:020000040000FA
:100000000002040000000000820E0000820E0000CA
:10001000820E0000820E0000820E0000820E0000A0
:10002000820E0000820E0000820E0000820E000090
:10003000820E0000820E0000820E0000820E000080
:10004000820E0000820E0000820E0000820E000070
:10005000820E0000820E0000820E0000820E000060
:10006000820E0000820E0000820E0000820E000050
:10007000820E0000820E0000820E0000820E000040
:10008000820E0000820E0000820E0000820E000030
:10009000820E0000820E0000820E0000820E000020
:1000A000820E0000820E0000820E0000820E000010
:1000B000820E0000820E0000820E0000820E000000
:1000C000820E0000820E0000820E0000820E0000F0
:1000D000820E0000820E0000820E0000820E0000E0
:1000E000820E0000820E0000820E0000820E0000D0
:1000F000820E0000820E0000820E0000820E0000C0
:10010000820E0000820E0000820E0000820E0000AF
:10011000820E0000820E0000820E0000820E00009F
:10012000820E0000820E0000820E0000820E00008F
:10013000820E0000820E0000820E0000820E00007F
:10014000820E0000820E0000820E0000820E00006F
:10015000820E0000820E0000820E0000820E00005F
:10016000820E0000820E0000820E0000820E00004F
:10017000820E0000820E0000820E0000820E00003F
:10018000820E0000820E0000820E0000820E00002F
:10019000820E0000820E0000820E0000820E00001F
:1001A000820E0000820E0000820E0000820E00000F
:1001B000820E0000820E0000820E0000820E0000FF
:1001C000820E0000820E0000820E0000820E0000EF
:1001D000820E0000820E0000820E0000820E0000DF
:1001E000820E0000820E0000820E0000820E0000CF
:1001F000820E0000820E0000820E0000820E0000BF
:10020000FFFFFF00FFFFFF00820E0000820E0000D4
:10021000820E0000820E0000820E0000820E00009E
:10022000820E0000820E0000820E0000820E00008E
:10023000820E0000820E0000820E0000820E00007E
:10024000820E0000820E0000820E0000820E00006E
:10025000820E0000820E0000820E0000820E00005E
:10026000820E0000820E0000820E0000820E00004E
:10027000820E0000820E0000820E0000820E00003E
:10028000820E0000820E0000820E0000820E00002E
:10029000820E0000820E0000820E0000820E00001E
:1002A000820E0000820E0000820E0000820E00000E
:1002B000820E0000820E0000820E0000820E0000FE
:1002C000820E0000820E0000820E0000820E0000EE
:1002D000820E0000820E0000820E0000820E0000DE
:1002E000820E0000820E0000820E0000820E0000CE
:1002F000820E0000820E0000820E0000820E0000BE
:10030000820E0000820E0000820E0000820E0000AD
:10031000820E0000820E0000820E0000820E00009D
:10032000820E0000820E0000820E0000820E00008D
:10033000820E0000820E0000820E0000820E00007D
:10034000820E0000820E0000820E0000820E00006D
:10035000820E0000820E0000820E0000820E00005D
:10036000820E0000820E0000820E0000820E00004D
:10037000820E0000820E0000820E0000820E00003D
:10038000820E0000820E0000820E0000820E00002D
:10039000820E0000820E0000820E0000820E00001D
:1003A000820E0000820E0000820E0000820E00000D
:1003B000820E0000820E0000820E0000820E0000FD
:1003C000820E0000820E0000820E0000820E0000ED
:1003D000820E0000820E0000820E0000820E0000DD
:1003E000820E0000820E0000820E0000820E0000CD
:1003F000820E0000820E0000820E0000820E0000BD
:100400000F802000007F2200000188000000000013
:100410000C00070000E82000010020001100070088
:10042000000020000000E000020032000000020096
:10043000000000004C0A0200000000000040DA004A
:100440000000FE004440A900C07B20000000E00046
:100450000300320000002000A00188004440A800F2
:100460000000060091018800800078000000EB0089
:1004700015003700E280400032A0B4009101BA00BC
:10048000E280400032A0B4009102BA00E280400055
:1004900032A0B4000002EB00472BDE00F507B200EB
:1004A000602CE10004003A000059EB008301E900F0
:1004B000FDFF3E00040037006128E100010032002A
:1004C0000082EB00040007001101BA000200E00006
:1004D000E8FF3A00000006003159BA008301E90044
:1004E0000C0032002159BA008301E90008003200F3
:1004F0000400E00003003A00E280400032A0B400B3
:10050000F5FF370011D9BA008301E900FAFF3A007C
:100510008100E800E180400032A0B4000000060045
:10052000202F00008CA9000042270000A9450000F0
:1005300007AE000042A7000037FE0000FF2F0000BA
:10054000F0FF00008860000019A90000CC22000024
:10055000A8C8000022A8000068A00000A9CC0000E4
:1005600002A90000C8020000000000000000000016
:1005700000000000AFCA000022370000A000000009
:10058000EB000000048000002635000080270000FA
:1005900036A80000A4060000A9A4000026A80000B8
:1005A000A4460000A9A4000066A90000A4860000DB
:1005B000A8C4000006A80000C4260000A9C40000CA
:1005C00046A90000C4660000A9C4000086A8000077
:1005D000C4220000A9C0000022EB0000800000003F
:1005E000202000000288000040110000A820000028
:1005F00062A8000021E20000A823000042070000DA
:1006000071000000B11000000C3200000900000071
:1006100020200000048800002011000020C00000FD
:100620000488000020110000204000000388000022
:100630002011000020B000000288000020110000FE
:100640003773000000200000400D000088200000EB
:100650001120000010000000882000001120000080
:10066000200000008820000011200000B0040000DD
:100670008820000011EB000000070000075C00006C
:100680000088000090010000075A000000B7000039
:1006900003E100000758000000B7000002E100007D
:1006A000BF02000081780000800200007800000096
:1006B00002070000530000007880000006070000D9
:1006C000510000007880000001200000028000003E
:1006D000074E00000078000000590000E983000088
:1006E000013A0000FCFF0000E00E000004320000B0
:1006F0000300000020E0000004880000201100003A
:1007000037E80000FF2A0000037C0000E10300003E
:10071000283E000010000000E0050000003A000044
:10072000120000002002000080B3000040C0000062
:100730007800000059B3000000C0000078000000FD
:1007400059B3000080CA00007800000059B30000CF
:1007500000C000007800000059B3000000C0000095
:100760007800000059B3000000C0000078000000CD
:100770005937000004000000EB800000002000005A
:10078000000500008820000011370000D1FF0000A4
:100790002002000080A700000D10000037020000BA
:1007A000002F0000F1FF000037CA0000FFA6000084
:1007B000010000003704000000BB0000850A0000B3
:1007C00024200000040700001A000000EB80000055
:1007D0000020000003040000BBB20000CABB000000
:1007E000B25A0000BBB200005AE9000083010000C9
:1007F0003AFB0000FF240000100000000711000079
:1008000000200000030400002002000080BA000065
:1008100014C00000E1320000043A000009000000AA
:10082000BA34000040E10000320400003A06000043
:1008300000BA000034400000E1320000043A000039
:1008400003000000E9830000013A0000F5FF00000A
:1008500037AE0000FF200000600500008820000087
:1008600011370000ADFF0000880000003B200000B1
:1008700050050000883000003B200000A00A000066
:10088000883000003BA8000061E700000000000085
:100890000000000000000000AF610000E73700002A
:1008A000FEFF000006000000002000001A0100000A
:1008B000EB80000005FE000000600000AE2200009A
:1008C00002370000030000008030000011470000E4
:1008D000000700000600000000E900008B05000092
:1008E0003AF80000FFE900000A0500003AF50000B0
:1008F000FF2000002F8C0000A608000000AE0000C2
:10090000CA220000376A0000FFA9000085600000CD
:10091000A985000080A9000023420000A921000051
:10092000E2EF000002210000A9C4000022A800009C
:10093000C02200008826000035880000273600000D
:10094000A9680000A0A80000C80200002000000064
:10095000008800006019000037490000FF2F0000E8
:10096000F8FF0000375A0000FF00000000080000F8
:1009700000C20000000000000000000000000000B5
:1009800000FE000000000000FFFF0000FFFF00006D
:10099000FFFF0000FFFF0000FFFF0000FFFF00005F
:1009A000FFFF0000FFFF0000FFFF0000FFFF00004F
:1009B000FFFF0000FFFF0000FFFF0000FFFF00003F
:1009C000FFFF0000FFFF0000FFFF0000FFFF00002F
:10110000FFFF0000FFFF000037B80000FE000000F6
:101110000304000000DF0000F90000007F3F000032
:101120000045000072610000736900006E670000F6
:10113000200000002E2E00002E0000002064000081
:101140006F6E0000650000005772000069740000B7
:10115000696E000067200000726F000077200000B9
:1011600000200000202000002055000070670000D3
:10117000726100006465000020630000616E000081
:10118000636500006C6C0000656400002E000000C8
:10119000646F00006E650000004500007261000091
:1011A000736900006E670000203000007830000096
:1011B00030300000302E00002E2E000000570000BE
:1011C00072690000746900006E6700002072000000
:1011D0006F770000203000002E2E00002E2000002F
:1011E0000053000075630000636500007373000026
:1011F00021000000557000006C6F00006164000069
:10120000206E000065770000206600006972000013
:101210006D770000617200006520000077690000B2
:1012200074680000207400006865000020640000FD
:1012300073330000302000004C6F00006164000038
:1012400065720000206100007070000020740000D2
:101250006F200000636F00006D7000006C6500007F
:1012600074650000207400006865000020750000AF
:101270007067000072610000646500002E000000CD
:10128000556E000069760000657200007361000011
:101290006C2000004453000033300000204C00005C
:1012A0006F6100006465000072200000696E00003C
:1012B00073740000616C00006C6500007220000017
:1012C000763000002E340000202800004329000062
:1012D00068720000697300002032000030310000A5
:1012E00030000000526500006C6500006173000072
:1012F00065640000207500006E64000065720000E7
:1013000020430000726500006174000069760000EF
:1013100065200000436F00006D6D00006F6E0000DF
:10132000732000006E7500006C6C0000206C0000E3
:1013300069630000656E0000736500002E00000008
:10134000466F0000756E000064200000626F0000B0
:101350006F7400006C6F0000616400006572000033
:101360002076000000200000756E00006B6E00000B
:101370006F7700006E20000028700000726F000080
:1013800062610000626C000079200000763200008B
:1013900029000000576900006C6C00002069000003
:1013A0006E730000746100006C6C0000206200002D
:1013B0006F6F0000746C00006F61000064650000D6
:1013C0007220000076000000547900007065000073
:1013D00020270000596500007327000020740000DA
:1013E0006F200000707200006F67000072610000E3
:1013F0006D20000074680000652000006E6500002C
:1014000077200000626F00006F7400006C6F0000B6
:1014100061640000657200002E0000004469000055
:10142000736300006F6E00006E650000637400005F
:10143000207000006F7700006572000020690000D6
:1014400066200000756E0000737500007265000074
:10145000202800006E6F000020680000617200000C
:101460006D200000646F00006E650000292E0000F2
:101470000030000031320000333400003536000007
:101480003738000039410000424300004445000065
:101490004630000078000000C400FA00EB000700AE
:1014A000C222A900B100070090C5B3009400070054
:1014B0000004E0002600320050C4B3009000070092
:1014C0000004E0002200320030C5B3008C000700A9
:1014D0000004E0001E003200008928001901070006
:1014E0000089280017010700C222A80010892800DF
:1014F000FE00070000402A0041010700A0892800E3
:10150000FA00070000802A00E1010700E0892800B6
:101510000C01070010892800F400070000802A0051
:1015200037010700A0892800F000070000802A008A
:10153000D7010700E089280002010700408A28003F
:10154000EA0007000000EB001007980026003700B3
:10155000108B2800FB00070000892800F900070015
:10156000D0FF37001E0090000043B0004901070083
:1015700000C2B300470107000000EB00000F780035
:101580000B0037001E0178009E009000000C200028
:101590000088B9009E00400000292800008040001B
:1015A0009040780064004700017178001E0FE80049
:1015B000F00B20009E0F1000F2FF34001E00900080
:1015C0004700DD008000780000802A000080400095
:1015D0008000780064004700B10107001E00900001
:1015E0000000E800100798001E009000E70F500070
:1015F000DCFF3400808C2800D2000700D08C28004B
:10160000BA0007000000EB00A1010700E0892800F4
:10161000CC000700F08D2800B40007000000EB00AC
:10162000000F7800050037001E017800E400470035
:1016300000C0EB0000F178001E0FE800F00B200066
:101640009E0F1000F8FF3400E400470040C0B300D4
:1016500080487800E40047000040EB00904098008C
:10166000E400470080CAB300A0409800E4004700AF
:101670000040EB00B0409800E40047000040EB0061
:10168000C0409800E40047000040EB00D0409800C4
:10169000640047008000EB0081010700808C280077
:1016A000A800070000892800A6000700108F280066
:1016B000A4000700A08F2800A200070023C2BF00DB
:1016C000614060000004E000FCFF320081BF2A009E
:1016D00001400100C222A800A0CFB300F70007001C
:1016E000A0CFB300F5000700C222A900A0CFB3002D
:1016F000F2000700A0CFB300F0000700F5FF3700AD
:101700000600FA002047980029010700004F7800E2
:101710001E407800DF00070000C6B3009E4F100097
:1017200007003600A0C7B3009E4F100004003E0023
:101730001E40780001CEB30001404000004F780009
:101740002E4090009E4F500003003A0010002000F1
:1017500020079800020037000000EB0020079800E7
:101760002E0090000080FA00000006000000FA0041
:10177000008928007300070000942800710007000A
:10178000008928006F000700209728006D000700DF
:10179000009A280055000700A0BF2A005601070044
:1017A000E10F400003003A00309B28004F00070083
:1017B0000C003700A0BF2A004F0107004800DE00E0
:1017C00004010700E0C2B300B2000700A0BF2A0076
:1017D0004901070080007800F00F200000806000C1
:1017E000FC0007000089280056000700A09C280084
:1017F0003E00070090882800104078000080FB0021
:10180000F4000700E0C2B300A200070080882800AF
:10181000104078000080FB00EE00070000892800DF
:10182000480007000089280046000700409E280065
:1018300044000700E0A028004200070000892800BB
:10184000400007000080FA00000006000000FA00D7
:101850004507A9000080EB00601988004227A90015
:10186000416A20009140780000CEB30000C06000C3
:101870005040B300A4E6B700416C200091407800CE
:1018800000CEB30000C060003040B300C4E6B70033
:10189000C922A800C902A800C8E2A800C8C2A800BE
:1018A000C942A800C222A900C022A900CB62A90097
:1018B000C962A900C002A900C202A900200220003A
:1018C000401188000000EB00001188002062A80091
:1018D0000000EB001011880021E2A8002342A800BC
:1018E0008560A9000080FA00000006000600FA00EA
:1018F00010079800020037001E40780065000700BE
:101900001E009000104F78001E407800404798005D
:101910004E4090000004E0000200320010C0B3000E
:10192000404798004E4090009E0090008100E800E3
:10193000110798000004E000EFFF3A000080FA0071
:10194000000006000600FA001007980002003700A9
:101950001E4078004F0007001E009000104F7800D6
:101960001E407800404798004E4090000004E00080
:101970000200320010C0B300404798004E40900073
:101980009E0090008100E800110798000004E0002C
:10199000EFFF3A00D0C0B3003E000700A0C0B30084
:1019A0003C0007000080FA00000006000400FA0076
:1019B0001007980090A42800CCFF07001E0090009C
:1019C0004400DE006F0F60009E00780090A32800A6
:1019D00000804000104078002E0007001E0090009C
:1019E0006F0F60009E00780090A3280000804000E8
:1019F00010407800270007000080FA000000060071
:101A00000400FA001007980090A42800B7FF070010
:101A10001E0090004C00DE006F0F60009E007800FA
:101A200090A32800008040001040780019000700B3
:101A30001E0090004800DE006F0F60009E007800DE
:101A400090A328000080400010407800110007009B
:101A50001E0090004400DE006F0F60009E007800C2
:101A600090A3280000804000104078000900070083
:101A70001E0090006F0F60009E00780090A3280069
:101A80000080400010407800020007000080FA004B
:101A9000000006000200FA00004F780023C2BF00D9
:101AA000624060000004E000FCFF3A001E00FB0002
:101AB000201188000080FA00000006000600FA00ED
:101AC000404798000040EB00204798000E00370088
:101AD0000000EB00000F780005003700A0CFB30036
:101AE0000F0007001E0078000000E800000F7800DB
:101AF0001E007800E30F5000F8FF36002E409000E3
:101B00000040E80020479800AE4090004E40900012
:101B100080CF5000EEFF39000080FA000000060080
:101B20000400FA00204798000040EB00004F7800C6
:101B3000130037000000000000000000000000005B
:101B40000000000000000000000000000000000095
:101B50000000000000000000000000000000000085
:101B60000000000000000000000000000000000075
:101B7000000000001E4078000040E800004F7800A0
:101B80009E4078002E40900080CF5000E9FF390041
:101B90000080FA00000006000000FA0022C2BF0028
:101BA000614060000080FB000080FA000000060039
:101BB0000000FA0022C2BF00614060000004E000A3
:101BC000FCFF3200301180000080FB000080FA0032
:101BD000000006000800FA00300798000040EB0003
:101BE000004F780000712200200798000040EB00B1
:101BF000104798001E0037003E0090002E01900014
:101C0000110009000280D800100798001E04E000AF
:101C100003003A001E0090000000E0000C003200BB
:101C20001E0090000043B0009AFF07009E00900045
:101C30002E0090000088B900800078003E009000DF
:101C4000010050003007980010C0B300004F78002A
:101C50002E009000A2002000110009000280D80090
:101C6000200798001E4090000040E80010479800B0
:101C70001E409000E34F5000DFFF36003E00900012
:101C80000043B00083FF07000080FA000000060058
:101C90000008BB00200424000C0007000000060020
:101CA000821F780002042000B0C8BB00B058BB00FF
:101CB000B058BB000201E900FBFF3A00100024000D
:101CC000020007004F01780000000600003B88007A
:101CD00050052000303B8800A00A2000303B8800DF
:101CE00061E7A800000000000000000061E7AF000D
:101CF000FEFF3700000006001000BA0000000600DA
:101D0000000000000000FE00FFFFFF00FFFFFF00DB
:101D1000FFFFFF00FFFFFF00FFFFFF00FFFFFF00CF
:101D2000FFFFFF00FFFFFF00FFFFFF00FFFFFF00BF
:101D3000FFFFFF00FFFFFF00FFFFFF00FFFFFF00AF
:101D4000FFFFFF00FFFFFF00FFFFFF00FFFFFF009F
:020000040001F9
:00000001FF
